:100000000EC07EC092C026C025C0C6C023C022C07C
:1000100021C020C01FC01EC08AC01CC01BC011242C
:100020001FBECFE5D2E0DEBFCDBF11E0A0E6B0E05D
:10003000EEE7F6E002C005900D92A230B107D9F7C5
:1000400021E0A2E0B1E001C01D92A233B207E1F7C6
:10005000A0D113C36BC0A895F89414BE91B5986154
:1000600091BD813031F0823031F082E481BD7894ED
:10007000089583E4FBCF87E4F9CFA895F89414BEE4
:1000800081B5886181BD11BC7894089585B7877E5C
:10009000806185BFF89485B7806285BF85B7846825
:1000A00085BF8B7F85BF7894889585B78F7D85BF09
:1000B00008950F931F93CF93DF938C01062E000CAE
:1000C000770B85E0660F771F8A95E1F760507040E7
:1000D00040E250E0C801A0D2E801005E1F4F8991C4
:1000E0008C3030F464E670E0F6D084E690E0CDD059
:1000F000C017D107A1F7DF91CF911F910F910895FC
:100100001F921FB61F9211248F93809104018111B9
:1001100007C010920301809127018F5F8093270110
:100120008F911F901FBE1F901895189518958F934B
:100130008FB78F93EF93FF93E2E0F1E081818460CA
:100140008183FF91EF918F918FBF8F9118958AB521
:1001500080688ABD8AB58F7B8ABD089582E089BF99
:1001600083E08ABD81E083BF12BE19BCB89A1092A9
:100170002F0110922C0110922E0110922D0110923D
:100180003101109230011092280110922901109231
:100190002A0110922B0108950F920FB60F921F9211
:1001A00011242F933F934F935F938F939F93AF931C
:1001B000BF93EF93FF9380912F0120912D013091F8
:1001C0002E01820F932F911D90932E0180932D016C
:1001D000E0912D01F0912E01349633E0F695E795EC
:1001E0003A95E1F7EF770E2E000CFF0BEE57FF4F1D
:1001F000808190912C01992309F445C020912C0114
:100200004091300150913101240F352F311D309331
:10021000310120933001E0913001F09131013496A9
:1002200093E0F695E7959A95E1F7EF770E2E000C9F
:10023000FF0BEE57FF4F9081890F96959695891B7E
:1002400089BD8091280190912901A0912A01B09146
:100250002B010196A11DB11D8093280190932901C6
:10026000A0932A01B0932B01FF91EF91BF91AF9121
:100270009F918F915F914F913F912F911F900F9080
:100280000FBE0F90189590E0D7CF109228011092D2
:10029000290110922A0110922B0125B7277E25BF34
:1002A0006FE070E094D1B0E0A0E04091280150915F
:1002B000290160912A0170912B0184179507A607E7
:1002C000B70708F4089525B7206225BF889525B79C
:1002D0002F7D25BFEACFCF93DF93EB011BBE8C3080
:1002E000F0F4E82FEE0FFF0BE659FF4F808180936B
:1002F0002F01818180932C012ADFCE01C6DF8AB5D0
:100300008F778ABD8AB58F7B8ABDC09810922F01E6
:1003100010922C0180E68BBFDF91CF910895863F2C
:1003200031F482E480932F0110922C01E5CF833FBA
:1003300011F481E2F7CF853FB1F482E280932F017F
:1003400010922C0104DFCE0163E070E051D1EB018B
:10035000CB019BDF8BE280932F01CE0196DF83E3FD
:1003600080932F01CACF843F51F683E380932F01FE
:1003700010922C01ECDECE0163E070E039D1EB018C
:10038000CB0183DF8BE280932F01CE017EDF82E2FF
:10039000E7CF90E896BD16BC88B3866088BB8BE03B
:1003A00080BD98B983E085BF80E68BBF86E085BBC2
:1003B000789481E050DE6ADE60DED0DE10920201C9
:1003C00081E08093040110920301109206011092C3
:1003D0000501E7E0F1E08FEF819391E0E732F90763
:1003E000D9F701E0D1E0CFEF13E026B3922F92705E
:1003F00021FB882780F980930401801709F4BEC08F
:10040000911122C0809103018160809303011092B9
:10041000270180E020DE3ADE009104018091030193
:1004200080FFB6C082E017DE31DE8091030182FFDB
:10043000DCCFD09302018A7F82608093030168EC55
:1004400070E083EF48DFD1CF109203018091270144
:100450009FEF980F9A3018F0C0932701DACF8A30B7
:1004600011F41092270181E0F6DD10DE06DE8091A6
:10047000020181111BC064E670E0809127012BDF2F
:1004800080910601803240F6E82FF0E0EE5FFE4FEB
:100490009091270195838F5F8093060140E250E0A1
:1004A00060EE70E087E091E0C7D0B6CF8130F1F424
:1004B000E091270164E670E08AE0E13029F0E23063
:1004C00029F464E670E08BE006DFA6CF67E0E33056
:1004D00049F00E2E000CFF0BE05AFF4F6081683090
:1004E00008F09ACF87E091E0E4DD96CF8230D9F42E
:1004F000E09127010E2E000CFF0BE05AFF4F808188
:1005000087FD0EC08093050110920601E7E0F1E03F
:10051000C19381E0E732F807D9F7109302017CCF4D
:100520001092020179CF833009F076CF80910601D5
:100530008032B0F01092020160E273E084EFCBDE13
:1005400060910501683008F067CF70E085E0660FC4
:10055000771F8A95E1F76050704040E250E0A2CFEB
:10056000E82FF0E0EE5FFE4F9091270195838F5FBB
:100570008093060164E670E083EFE1CF992309F4EC
:100580004BCF1092020110920301C093270144CF78
:1005900081FF11C082E05FDD79DD8091030182FF80
:1005A00024CF92E090930201897F8093030168EC4D
:1005B00070E085EF47CF85B7877E806185BF85B7BF
:1005C000806285BF889585B78F7D85BF0ECF00245B
:1005D000552704C0080E591F880F991F009729F04E
:1005E00076956795B8F37105B9F7802D952F089525
:1005F000AA1BBB1B51E107C0AA1FBB1FA617B70749
:1006000010F0A61BB70B881F991F5A95A9F7809564
:100610009095BC01CD010895DC01CB01FC01E1996D
:10062000FECF06C0FFBBEEBBE09A31960DB20D9235
:1006300041505040B8F70895DC01A40FB51F415058
:10064000504040F0CB01840F951F2E9105D04150B2
:100650005040D8F70895262FE199FECF9FBB8EBB5F
:10066000E09A01970DB2021639F01CBA2DBB0FB6F5
:0E067000F894E29AE19A0FBE0895F894FFCF35
:10067E0000FFFFFF010203040506573D4F2E572EC4
:10068E00602E4F32573260324F38573860384F3DF8
:10069E00603D404346494C4F5255585B5E60636621
:1006AE00686A6D6F7173757678797B7C7D7E7E7FDF
:1006BE007F7F7F7F7F7F7E7E7D7C7B797876757373
:1006CE00716F6D6A686663605E5B5855524F4C4938
:1006DE004643403C393633302D2A2724211F1C191E
:1006EE00171512100E0C0A09070604030201010069
:1006FE0000000000000001010203040607090A0CB5
:10070E000E10121517191C1F2124272A2D303336CF
:02071E00393C64
:00000001FF
